:1000000070C100008BC1000089C1000087C10000E1
:1000100085C1000083C1000081C100007FC10000D4
:100020007DC100007BC1000079C100000C9429094A
:1000300075C1000073C1000071C10000CBC6000093
:100040006DC100006BC1000069C100005DC7000008
:1000500065C1000063C1000061C100005FC1000014
:100060005DC100005BC1000059C1000057C1000024
:1000700055C10000CA1006110C1113111B112411D7
:100080003611451109121F12241229122E1239128B
:100090003E1248124E1255125B126012681265022F
:1000A000700276027C02840289029002CF02EB0287
:1000B000FC020603120326032A032F031405370547
:1000C000C8063705C8067E05A005C8068B069E062D
:1000D0005A0D5F0D6C0D760D850D8C0DC80D6D0ED6
:1000E0006D0ED80DE80DFC0D070E140E280E300E07
:1000F000590E302E392E300005010980A1018501ED
:100100001981298315002501950375018102950147
:1001100075058101C0050C0901A101850209B0091D
:10012000B109B209B309B409B509B609B709B809E3
:10013000CD09E209E909EA0A8A010A92010A940151
:100140000A21020A23020A24020A25020A27020AB5
:100150002A02150025019516750181029501750287
:100160008101C005010906A101050819012903152E
:100170000025019503750191029501750591010511
:100180000719E029E7150025019508750181020589
:100190000719002931150025019532750181029555
:1001A000017501810105071933299B15002501956A
:1001B00069750181029501750181010507199D2964
:1001C000A41500250195087501810295017503812B
:1001D00001C00600FF0901A1010902150025FF75F4
:1001E00008950881020903150025FF7508950891F7
:1001F00002C005010906A10175019508810195015B
:1002000075088101950575019101950175039101AD
:10021000950675088101C009026D00040100A03235
:10022000090400000103010100092111010001225C
:1002300025000705810308000A09040100010300E5
:100240000000092111010001222000070583030895
:10025000000509040200010300000009211101004A
:1002600001226F0007058203200001090403000139
:1002700003000000092111010001226B0007058421
:100280000308000A1201100100000020810402008E
:100290000100010200012203690062006D002D00CF
:1002A000630061007000730065006E0073006500FC
:1002B0002D007500730062000000220354006F00DF
:1002C0006D00200057006F006E0067002D00430096
:1002D0006F0072006E0061006C006C00000004038F
:1002E000090411241FBECFEFD4E0DEBFCDBF11E063
:1002F000A0E0B1E0E6E1F7E202C005900D92A03681
:10030000B107D9F713E0A0E6B1E001C01D92AD330B
:10031000B107E1F70E94E40E0C94891371CEEF92BD
:10032000FF920F931F93CF93DF938C0191E0EE2404
:10033000E394F12C461720F120E030E0A62FB0E046
:10034000AA0FBB1FAA0FBB1FE801C90FD11DFD01DA
:10035000E20FF31FE75AFD4F808183304CF0888114
:10036000F701022E01C0EE0F0A94EAF7E82BE883AA
:100370002F5F3F4F2430310551F76F5F9F5FDACF1A
:10038000DF91CF911F910F91FF90EF9008952498E6
:100390002598269827982C982D982E982F9810926B
:1003A000B6021092B50280912603823019F4249A85
:1003B000259A269A08959C0128553240283A3140C2
:1003C00010F40C94771308959093BE028093BD02AD
:1003D0002898880F991F880F991F9EBD0DB407FE9E
:1003E000FDCF9EB58EBD0DB407FEFDCF8EB5289A0C
:1003F0000895AF92BF92CF92DF92EF92FF920F9348
:100400001F93CF93DF93E901D80121E08533920751
:1004100009F040C080910301882309F44EC1109275
:10042000030190913E01911148C168E3E62E62E01C
:10043000F62E60E0F7012081222301F120E030E078
:100440007CEF790FF701408150E0022E02C05595F4
:1004500047950A94E2F740FF0CC0192F120F472F5F
:10046000420F413A30F4AE01460F511DFA0112839A
:100470006F5F2F5F3F4F2830310521F7FFEFEF1AF5
:10048000FF0A985F983AB1F690915402988328E059
:1004900030E03DC121E08532920709F010C1209182
:1004A0003E0188E0FE0111928A95E9F7E0912A0366
:1004B000E8838E2F90E0FC013197EF30F10508F0D2
:1004C000F7C0E15BFF4F0C942D1384E0898398E023
:1004D0009A8397E19B838C8381E08D832E839FC0D9
:1004E00046E060E0CE011BDF83E00BC04DE067E03B
:1004F000CE0115DF84E005C044E16EE0CE010FDFE0
:1005000085E080932A03D4C047E165E1CE0107DF8F
:1005100086C09091BD028091BE0299838A837FC07C
:10052000E0901B03F0906101FE1411F08F2D05D6B1
:10053000909160018F2D8295880F880F807C892B88
:1005400089832296692F70E0660F771F660F771FE9
:1005500040E050E0FA01E60FF71FE154FD4F8081C3
:1005600089934F5F5F4F44305105A1F79F5F9731EB
:1005700019F0909360010BC01092600191E09F0D03
:10058000943019F09093610102C010926101809142
:1005900061018E1509F48CC08E2DCFD589C0809154
:1005A00062018983E82FF0E0EE0FFF1FEE0FFF1FBF
:1005B000E45EFC4F40815181628173814A835B8399
:1005C0006C837D838F5F823019F08093620170C0ED
:1005D000109262016DC0DE011196E2EFF0E081E061
:1005E0008F5F94919D93992319F031968730C1F7CD
:1005F000C80FD11D188213C0809126038983809172
:1006000025038A83809124038B8309C0809127036B
:1006100090912803A091290389839A83AB83109238
:100620002A0346C060916301698370E0660F771FFB
:10063000660F771F44E050E0CE0102960E945013EF
:10064000809163018F5F8093630132C01982809132
:10065000580203C088EA898381E08A8329C0F09028
:1006600064018F2D90E08A569F4F880F991F880F45
:10067000991FF98222965C01F4E0AF0EB11C81153E
:1006800024E0920738F081E08F0D8A3678F4809369
:1006900064010EC06C01EFEFCE1ADE0A0E946013F7
:1006A0008993CA14DB0479F3C601E9CF109264017F
:1006B00088E090E0F8019183808380E081C0F1E0E0
:1006C00085319F0739F5809104018823B1F3109299
:1006D000040180913E01882381F39E012F5F3F4FEB
:1006E00068E372E095E1960FFB014191BF01F901CA
:1006F00041939F019613F8CF9981907F99839D89AB
:100700009F719D8B90915402988326E130E02D9348
:100710003C9356C08550914081F6FB01808188232F
:1007200019F08093000104C080910001FB018083D7
:10073000809100018130D9F480910201882309F46D
:10074000BCCF1092020190914C02929596959770B1
:10075000988320916501291719F09093650101C0D4
:1007600080E021E030E02D933C9392E027C082307E
:1007700009F0A3CF80910101882309F49ECF109244
:10078000010180914D02888380914E02898380917E
:100790004F028F738A83E6E6F1E080E023E02E0FBC
:1007A00099913081391711F0908381E031962E13A1
:1007B000F7CF23E030E02D933C9391E0909300013C
:1007C000DF91CF911F910F91FF90EF90DF90CF902D
:1007D000BF90AF9008952091E4003091E50095E638
:1007E0004091EC00842F817040FF22C08091E8008E
:1007F00080FD1CC080913403882391F0853091F0F6
:100800008091EB0085FD10C04091E4005091E5001F
:100810004217530729F39A01915011F784E0089584
:1008200082E0089583E0089581E0089580E00895CE
:100830004091E80042FFDECF089580912C0387FFAE
:1008400011C08091E80082FD05C0809134038111C0
:10085000F8CF11C08091E8008B770BC080913403F2
:10086000882349F08091E80080FFF8CF8091E8006C
:100870008E778093E8000895982F953058F59093DF
:10088000E900981739F07091EC002091ED0050913B
:10089000F00003C0242F762F50E021FF19C03091C3
:1008A000EB003E7F3093EB003091ED003D7F3093C5
:1008B000ED003091EB0031603093EB007093EC0071
:1008C0002093ED005093F0002091EE0027FF07C029
:1008D0009F5FD3CF8F708093E90081E0089580E01F
:1008E000089520913203309133032617370748F0DB
:1008F0006115710539F42091E8002E772093E80006
:1009000001C0B90140E06115710581F12091340306
:100910002223E9F12530E9F12091E80023FD35C0DB
:100920002091E80022FD2BC02091E80020FFEBCFB2
:100930002091F20030E0FC01CF016115710559F002
:100940002032310540F481918093F10061507109AA
:100950002F5F3F4FF1CF41E02032310509F040E0F9
:100960002091E8002E772093E800CDCF4111CECF23
:1009700006C080913403882351F0853051F0809176
:10098000E80082FFF6CF80E0089581E0089582E0DC
:10099000089583E008950F931F93CF93DF93CDB70E
:1009A000DEB7AA970FB6F894DEBF0FBECDBF809119
:1009B0003403882309F403C21091E9001F70909159
:1009C000EC00892F817090FD80E8182B1092E900CF
:1009D0008091E80083FFEAC1ECE2F3E088E08E0F4B
:1009E0009091F10091938E13FBCF85E391E063D753
:1009F00085E291E060D785E191E05DD785E091E007
:100A00005AD78091E80083FFC3C180912C03909155
:100A10002D03492F50E04A30510508F0B9C1FA01C1
:100A2000E25AFF4F0C942D13803881F0823809F080
:100A3000AFC1809130038F708093E9008091EB000B
:100A400085FB882780F91092E90007C08091B802E1
:100A5000882311F082E001C080E09091E800977F48
:100A60009093E8008093F1001092F10060C1282F6C
:100A70002D7F09F08DC1882319F0823061F088C183
:100A800080912E03813009F083C1933009F080E01A
:100A90008093B8022DC080912E03811129C08091CE
:100AA00030038F7009F474C18093E9009091EB00DA
:100AB00090FF1EC090912D03933021F48091EB00A4
:100AC000806214C09091EB0090619093EB0021E064
:100AD00030E0A90102C0440F551F8A95E2F7409308
:100AE000EA001092EA008091EB0088608093EB00AE
:100AF0001092E9008091E800877F1CC1811148C1F4
:100B000000912E030F778091E3008078802B8093F3
:100B1000E3008091E800877F8093E8008EDE80917B
:100B2000E80080FFFCCF8091E30080688093E300C1
:100B3000011102C082E001C083E08093340328C128
:100B40008058823008F024C180912E0390912F03A9
:100B50008C3D53E0950771F583E08A838AE28983AF
:100B60004FB7F894DE01139620E03EE051E2E32F08
:100B7000F0E050935700E49120FF03C0E295EF703E
:100B80003F5FEF708E2F90E0EA3010F0C79601C003
:100B9000C0968D939D932F5F243149F74FBF80916D
:100BA000E800877F8093E8006AE270E0CE0101965A
:100BB00098DEABC0E0913003292F33272330310575
:100BC000A9F06CF42130310509F4F4C0223031056C
:100BD00009F0DEC08DE690E0E7E1F2E04CC02132A2
:100BE000310531F12232310589F1D2C099278130A6
:100BF000910571F08230910599F0892B09F0C8C0F8
:100C0000EEEDF2E0E4918E2F90E0EEEDF2E030C0F8
:100C1000EAEBF2E0E4918E2F90E0EAEBF2E028C0FC
:100C2000E6E9F2E0E4918E2F90E0E6E9F2E020C000
:100C3000E43008F0ADC0F0E0EE0FFF1FEF5AFE4FBA
:100C40000190F081E02D89E090E015C0E43008F0DB
:100C50009FC08E2F90E0FC01EE0FFF1FE75BFE4F61
:100C60000190F081E02DDC01AB5BBE4F8C9190E0F8
:100C7000009709F48DC02091E800277F2093E800B9
:100C800020913203309133032817390708F4C90142
:100C900040E0009769F1209134032223B1F125301F
:100CA000A1F12091E80023FD30C02091E80022FD51
:100CB00028C02091E80020FFECCF2091F20030E026
:100CC000009759F02032310540F444914093F100EF
:100CD000319601972F5F3F4FF3CF41E0203231052E
:100CE00009F040E02091E8002E772093E800D1CF72
:100CF0004111D1CF06C080913403882331F0853073
:100D000021F08091E80082FFF6CF8091E8008B7798
:100D10008093E8003DC0803809F03AC08091E80037
:100D2000877F8093E8008091B9028093F1008091E1
:100D3000E8008E778093E80080DD2AC0811128C00A
:100D400000912E03023020F58091E800877F809388
:100D5000E8000093B90271DD011106C08091E30043
:100D600087FD02C081E001C084E08093340385E305
:100D700091E062D585E291E05FD585E191E05CD5B7
:100D800085E091E059D58091E20084608093E20093
:100D90008091E80083FF0AC08091E800877F8093FC
:100DA000E8008091EB0080628093EB001F7010934D
:100DB000E90005C082E190E0E4E8F2E05CCFAA96A9
:100DC0000FB6F894DEBF0FBECDBFDF91CF911F915C
:100DD0000F9108951F920F920FB60F9211242F9327
:100DE0003F934F935F938F939F93AF93BF93EF93F3
:100DF000FF93CF93DF9300D000D0CDB7DEB7198239
:100E00001A821B821C828091BB02873118F046989F
:100E100088E137C0489B02C091E09983499B02C09A
:100E200091E09A834A9B02C091E09B834B9B02C056
:100E300091E09C83DE01119620E030E090E0880F85
:100E4000991F880F991F57E04D91FC01E20FF31F86
:100E5000E75AFD4F442341F0408141504083408197
:100E600043304CF4108207C040814F5F4083408183
:100E700043300CF050832F5F3F4F2430310521F772
:100E8000C6CF459A45988150E1F7469A8091BB02BA
:100E900097E18F5F873130F0809158028F5F8093A8
:100EA000580280E0E82FE695E695E695F0E0E95DEA
:100EB000FC4F208130E0482F477002C035952795C0
:100EC0004A95E2F720FF03C0915019F787E180931C
:100ED000BB021092810010928500109284000F9046
:100EE0000F900F900F90DF91CF91FF91EF91BF91F5
:100EF000AF919F918F915F914F913F912F910F9063
:100F00000FBE0F901F9018951F920F920FB60F9261
:100F100011248F939F934698449A459A45984498F4
:100F200080E09091BB02891720F4459A45988F5F25
:100F3000F8CF469A82E0809381009F918F910F9025
:100F40000FBE0F901F901895EEE6F0E080818D7F28
:100F50008083EFE6F0E080818D7F808315BC109266
:100F600081008CE5E9E5F2E0DF011D928A95E9F761
:100F7000089584B5826084BD89E187BDEEE6F0E026
:100F800080818260808385B5836085BD10928000FA
:100F900088E090E09093890080938800EFE6F0E08D
:100FA000808182608083089580915702992787FD10
:100FB000909565E070E00E9408138A569E4FFC01F0
:100FC0008081E82FE695E695E695F0E0E85CFD4F38
:100FD000282F277081E090E0022E01C0880F0A942C
:100FE000EAF7809590818923808308958093570242
:100FF0008FEF809356021092B7021092BC0281E0EC
:1010000080935502D1DF8091540280933702809300
:101010003602089590919501191674F420915602A4
:10102000280F20935602981B97FD03C090939501BB
:1010300014C01092950111C09091940119166CF48E
:1010400020915602280F20935602981B97FD03C04B
:101050009093940102C01092940181E08093550214
:1010600008959F92AF92BF92CF92DF92EF92FF923C
:101070000F931F93CF93DF938FEF80939301809310
:1010800057021092360286E9C82E81E0D82E00E081
:1010900010E0C8E5D2E095E0992EF601292D1192D5
:1010A0002A95E9F7CE0106968115944078F5CE0190
:1010B0000E9460139FEF980F9E3F40F5F601D48386
:1010C000C3838083CE0101960E94601398012A5643
:1010D0003E4F5901F90181837E01F3E0EF0EF11CCF
:1010E000CE0102960E946013F5018283C7010E941F
:1010F0006013B82ECE0104960E946013C82FD0E072
:10110000CB0DD11D2296CE0DDF1D02C0C0E0D4E074
:10111000F5E0CF0ED11C0B5F1F4F003A110509F00F
:10112000BCCFDF91CF911F910F91FF90EF90DF9097
:10113000CF90BF90AF909F900895AF92BF92DF92F3
:10114000EF92FF920F931F93CF93DF93D82EEFEF81
:10115000E80FE33040F4F0E0EE0FFF1FE75AFE4FD8
:10116000A080B18003C082E0A82EB12C00E010E086
:10117000C0E0D0E07E01E00EF11EC5018E0D9F1D86
:101180000E9460138F3F09F480E0F701E154FD4FA6
:1011900080832196C430D10569F70C5F1F4F0C3551
:1011A000110531F7D0921B03DF91CF911F910F9161
:1011B000FF90EF90DF90BF90AF90089583B185FBD3
:1011C000882780F991E08927089590912B03962331
:1011D000811102C031F402C0992319F01092BA02B1
:1011E0001CC08091BA0291E0980F9093BA028111CD
:1011F00014C0E42FE695E695E695F0E0E85CFD4F37
:10120000477081E090E0042E01C0880F0A94EAF74D
:101210009081892B808381E0089580E008958AE79A
:1012200091E00E9460138F3018F480932603089594
:10123000109226030895ABD880912603813029F0BF
:1012400038F083508C3020F42D9A269A279A2F9AC2
:1012500008951F920F920FB60F9211242F933F9370
:101260004F935F936F937F938F939F93AF93BF93AE
:10127000EF93FF938091E10082FF72C08091E200C2
:1012800082FF6EC08091E1008B7F8093E1008091AE
:10129000430190914401009729F0019790934401F4
:1012A000809343018091330190913401009729F09C
:1012B00001979093340180933301809123019091A1
:1012C0002401009729F00197909324018093230132
:1012D0008091130190911401009729F00197909348
:1012E0001401809313018091B6028F3F19F08F5F34
:1012F0008093B60280912603813021F000F1835063
:101300008C30E8F49091B60280912503981302C0C6
:101310002E9815C020912403921303C083E085BD4D
:101320000EC08091B502882351F0291740F4109225
:10133000B60281508093B5022E9A15BC16BC8091DE
:10134000B702882369F09091BC029F5F9A3019F030
:101350009093BC0205C01092BC0281508093B702EA
:101360008091E10080FF18C08091E20080FF14C0EE
:101370008091E2008E7F8093E2008091E2008061A4
:101380008093E2008091D80080628093D80019BCDD
:10139000109234030E94C7018091E10084FF2DC0A8
:1013A0008091E20084FF29C084E089BD86E089BD88
:1013B00009B400FEFDCF8091D8008F7D8093D800C6
:1013C0008091E1008F7E8093E1008091E2008F7E2A
:1013D0008093E2008091E20081608093E20080913E
:1013E000B902811106C08091E30087FD02C081E04F
:1013F00001C084E0809334031EDF8091E10083FF0D
:1014000024C08091E20083FF20C08091E100877FAB
:101410008093E10082E0809334031092B9028091BE
:10142000E1008E7F8093E1008091E2008E7F8093C7
:10143000E2008091E20080618093E20042E260E09D
:1014400080E01ADA81E080933E01FF91EF91BF9135
:10145000AF919F918F917F916F915F914F913F914C
:101460002F910F900FBE0F901F901895AF92BF92C3
:10147000CF92DF92EF92FF920F931F93CF93DF9360
:10148000B0901B0380E059DE4FEB52E080E0A12CCE
:10149000D12CE82FE695E695E695F0E0E95DFC4F66
:1014A000208130E0982F977002C0359527959A9546
:1014B000E2F720FD12C020E030E0FA01E20FF31F56
:1014C0009081992329F0913011F4A39401C0D39411
:1014D0002F5F3F4F2430310581F78F5F4C5F5F4FA7
:1014E0008731B9F6C0E0D0E0EE24EA9493E0F92E1B
:1014F00000E010E0C701801B910B8230910508F4D9
:101500004CC0EC01D695C795C00FD11FCE010E94EB
:10151000E40110925802809158028431E0F34FEBBD
:1015200052E020E030E0A0E0E22FE695E695E69577
:10153000F0E0E95DFC4F808190E0622F677002C0AF
:10154000959587956A95E2F780FD1AC080E090E056
:10155000B901660F771F660F771FFB01E80FF91FB0
:10156000E75AFD4FE081E3303CF4FA01E80FF91F40
:10157000E081E23008F0AF5F01968430910569F7B1
:101580002F5F3F4F4C5F5F4F2731310569F6AD1537
:1015900010F08E01AFCF7E01ADCF8E01CC24CA9466
:1015A000A3E0DA2EE12CF12CC6018E199F098230BE
:1015B000910508F44CC0EC01D695C795CE0DDF1D02
:1015C000CE010E94E40110925802809158028431A9
:1015D000E0F38FEB92E020E030E0A0E0E22FE69530
:1015E000E695E695F0E0E95DFC4F408150E0622F22
:1015F000677002C0559547956A95E2F740FD1BC09C
:1016000040E050E0B901660F771F660F771FFB01BE
:10161000E40FF51FE75AFD4FE081E3303CF0FC0199
:10162000E40FF51FE081E13009F4AF5F4F5F5F4FDA
:101630004430510561F72F5F3F4F04962731310544
:1016400069F6AA1510F06E01AFCF7E01ADCFC801CB
:101650008C1B9D0B63E070E0ECD7CB018C0F9D1FC2
:101660000E94E401E8DD8B2DDF91CF911F910F9156
:10167000FF90EF90DF90CF90BF90AF905ECD2F9214
:101680003F924F925F926F927F928F929F92AF9212
:10169000BF92CF92DF92EF92FF920F931F93CF935F
:1016A000DF9300D01F92CDB7DEB77C014DB65EB69A
:1016B00080913403843009F0A4C08091E4009091BB
:1016C000E500F701228533852817390709F499C009
:1016D00081818F708093E9008091E80085FF91C03F
:1016E0008DB69EB6408550E08DB79EB7841B950B96
:1016F0000FB6F8949EBF0FBE8DBFEDB7FEB7319603
:101700006F015F011B821A82198260E070E0CF01D5
:10171000C0D78E010F5F1F4F960140E0BE016D5F85
:101720007F4FC7010E94F901282EF7018485958516
:10173000892B51F091E080E026853785232B09F035
:1017400090E0092F182F02C000E010E0F70166803A
:1017500077806114710489F049815A81B301C6010F
:1017600082D733243394892B09F4312CF701408537
:1017700050E0B601C30184D701C0312C89819A8120
:10178000892B99F1211004C0311002C0012B69F19D
:10179000F701848595859787868781818F708093EF
:1017A000E9008B8181118093F10009811A8113D89E
:1017B000882369F08091E8008E778093E80015C057
:1017C000F50181915F018093F1000150110901152C
:1017D000110581F38091E80085FDF2CF8091E8004A
:1017E0008E778093E800D7D8E2CF8091E400909183
:1017F000E500F701938782870FB6F8949EBE0FBE6F
:101800008DBE0FB6F8945EBE0FBE4DBE0F900F900A
:101810000F90DF91CF911F910F91FF90EF90DF908C
:10182000CF90BF90AF909F908F907F906F905F9080
:101830004F903F902F900895CF93DF93FC01DC01F0
:10184000199687E0ED0119928A95E9F781E0818781
:1018500084EF91E09587848783E0848361816111BF
:1018600002C081E025C095810280F381E02D862FA2
:101870008F70853010F080E01BC0923010F442E091
:1018800001C046E028E030E090E02E173F0720F44A
:101890009F5F220F331FF9CF9295907F492B661FD0
:1018A0006627661F606C0E943C048111DACFE3CF8B
:1018B000DF91CF9108958F929F92AF92BF92CF9276
:1018C000DF92EF92FF920F931F93CF93DF9300D09D
:1018D0001F92CDB7DEB76C01EDB6FEB68091E80081
:1018E00083FF5DC2F601808190E02091300330914A
:1018F00031032817390709F052C280912D03833034
:1019000009F4F1C130F4813071F0823009F42AC257
:1019100046C28A3009F40DC28B3009F4F5C1893012
:1019200009F03DC24FC080912C03813A09F037C2C3
:101930008DB69EB61A82198280912E0310912F03C4
:101940008B83F6018085482F50E08DB79EB7841BAE
:10195000950B0FB6F8949EBF0FBE8DBFEDB7FEB7C7
:1019600031965F0160E070E0CF0193D64FEF410FF9
:101970008E010F5F1F4F9501BE016D5F7F4FC60146
:101980000E94F901F60186819781009721F0408538
:1019900050E0B50175D61092E9008091E800877F8C
:1019A0008093E80069817A81C5010E947104809169
:1019B000E8008B778093E8000FB6F8949EBE0FBEC8
:1019C0008DBEEDC180912C03813209F0E8C10DB7C5
:1019D0001EB7409132035091330330912E038DB7DF
:1019E0009EB7841B950B0FB6F8949EBF0FBE8DBF9C
:1019F00001962091E800277F2093E80041155105CA
:101A000029F42091E8002B772093E800FC01411590
:101A1000510521F120913403222321F1253011F1C8
:101A20002091E80023FD1EC02091E80022FFEFCFA7
:101A30002091F200222331F02091F10021934150B6
:101A40005109B1F72091E8002B772093E800DFCF10
:101A500020913403222331F0253021F02091E80039
:101A600020FFF6CF2091E8002E772093E800A1E038
:101A7000B0E0311102C0A0E0B0E0E5E3CE16E1E055
:101A8000DE0629F420913E01211127C121C1F5E292
:101A9000CF16F1E0DF0609F012C1A80FB91FEC91D3
:101AA0004E2F50E04131510508F017C1FA01E859B5
:101AB000FF4FD3C511968C9180932A030EC11196C6
:101AC0002C91119712968C9190E0982F8827820F75
:101AD000911D0E94E40101C111968C91882309F4A3
:101AE000FCC032DAE0E0F8E10995F7C011968C917C
:101AF000882309F4F2C06091BD0280E090E0F7D540
:101B00006091BE0281E090E0A1C011968C91882383
:101B100009F4E3C0ABDCE1C013966C911397129605
:101B20002C91129711969C91492F4F7392959695EF
:101B300096959370473108F0D0C0243008F0CDC09E
:101B4000EFEFE90FE33040F4F0E0EE0FFF1FE75A4C
:101B5000FE4FA081B18102C0A2E0B0E080911B03E2
:101B600030E050E098130AC0FA01EE0FFF1FEE0FAD
:101B7000FF1FE20FF31FE154FD4F6083CA01880F7E
:101B8000991F880F991F820F931F8A0F9B1F5EC09A
:101B900012966C91129711968C91883008F09DC026
:101BA00090E0FC01E45EFC4F60838E589E4F4EC077
:101BB00013968C91139712969C91129711962C91D3
:101BC00020932603909325038093240334DB85C060
:101BD00011968C91882309F480C0609126038AE7CE
:101BE00091E085D5609125038BE791E080D56091E8
:101BF00024038CE791E02AC011968D919D91AC91C0
:101C00008093270390932803A093290366C011961D
:101C10008C91882309F461C043E050E06DE771E0E6
:101C200087E293E055D559C013966C91139712969D
:101C30008C91129790E0982F882711962C91820F03
:101C4000911D8115F4E09F0708F047C050D545C0AD
:101C500011968C91882311F08CD93FC075D93DC065
:101C60001596BC9015971496AC90149713969C906B
:101C700013971196CC901197D12C26E9C20ED11C46
:101C8000CC0CDD1CCC0CDD1C12966C91C6010E94A4
:101C9000DB01692DC60101960E94DB016A2DC60198
:101CA00002960E94DB016B2DC60103960E94DB01A8
:101CB00014C011968C91882381F0D3D90EC0E5E130
:101CC000CE16E1E0DE0649F420913E01222329F000
:101CD000A80FB91F8C9180932B030FB6F8941EBFE9
:101CE0000FBE0DBF5CC080912C03813A09F057C034
:101CF0008091E800877F8093E8008091E80080FF72
:101D0000FCCFF601818542C080912C03813209F01D
:101D100046C08091E800877F8093E8000E941D0400
:101D200090912E0381E0911101C080E0F60181873E
:101D300036C080912C03813291F58091E800877F35
:101D40008093E8000E941D0480912E0390912F0340
:101D5000882736E0969587953A95E1F7F6019587BD
:101D600084871DC080912C03813AC9F48091E800DA
:101D7000877F8093E8008091E80080FFFCCFF60128
:101D80008485958596958795969587958093F1009E
:101D90008091E8008E778093E8000E941D040FB6C2
:101DA000F894FEBE0FBEEDBE0F900F900F90DF9126
:101DB000CF911F910F91FF90EF90DF90CF90BF9048
:101DC000AF909F908F900895CF93DF931F92CDB7E0
:101DD000DEB784B7877F84BF88E10FB6F89480931D
:101DE0006000109260000FBE90E080E80FB6F8949B
:101DF00080936100909361000FBE219A209A229AED
:101E000084E58CBD8DB581608DBD289A3C9A3D9A44
:101E10003E9A88E1459A45988150E1F7469A80912B
:101E200063008E7F8093630081E08093690110924C
:101E3000E2001092E1008091D8008F778093D80063
:101E40008091D80080688093D8008091D8008F7DE1
:101E50008093D80084E089BD86E089BD09B400FE86
:101E6000FDCF109234031092B9021092B80242E2F0
:101E700060E080E00E943C048091E1008E7F8093CE
:101E8000E1008091E20081608093E2008091E200B5
:101E900088608093E2008091E0008E7F8093E00074
:101EA000789443E050E06DE771E087E293E0F8D387
:101EB000809127038F3F71F4809128038F3F51F465
:101EC000809129038F3F31F4109227031092280349
:101ED000109229038CE5E9E5F2E0DF011D928A9575
:101EE000E9F71092750180E028D948E050E062E7F8
:101EF00071E08CE193E0D4D3B4D891D98BE791E031
:101F0000DFD3809325038CE791E0DAD38093240319
:101F1000EFE1FEE43197F1F700C000002AD881E03C
:101F200090E0CED390E0182F002780E090E0C8D357
:101F30009801282BC9010E94E4018091BD02909173
:101F4000BE02019609F492DA88E392E0FDE1BF2E29
:101F5000B80E01E010E086E791E0ADE1AA2EA80EF0
:101F60008CE193E0B8E09B2E980E80913E0188238F
:101F700019F08091040102C0809103018111F3C224
:101F800076E7C72E71E0D72EE8E3EE2EE2E0FE2ED4
:101F9000F701D60180818D931192BE12FBCF40E0F4
:101FA00050E020E030E0C901880F991F880F991F89
:101FB000840F951FFC01E75AFD4F60816330C4F028
:101FC000FC01E154FD4F8081883E90F4E82FE695B6
:101FD000E695E695F0E0E85CFD4F8770B80102C039
:101FE000660F771F8A95E2F7CB019081892B80835A
:101FF0002F5F3F4F27313105B1F64F5F5F4F4430C0
:10200000510579F6A8E3B2E0E6E7F1E091918D9110
:10201000981304C0AE12FACF812C02C08824839496
:10202000E091570230913602EF3F09F44CC1FF278F
:10203000E7FDF095CF0165E070E0EAD28A569E4F49
:10204000DC0113964D905C9014978091540290910E
:102050003702292F20952823232B9095982B922304
:10206000909336028093370270905602BFEF7B1236
:102070000AC0C201039624D3809395017092940103
:102080001092560221C08091950181113FC080912C
:1020900094018F3F69F5CF0165E070E0B9D28A56AF
:1020A0009E4FFC012081E22FE695E695E695F0E053
:1020B000E85CFD4F808190E0277002C09595879580
:1020C0002A95E2F780FF03C00E94D4074EC1C201E7
:1020D0000496F6D28093940187FF07C091E0909315
:1020E00074018F778093940140C1109274013DC1B7
:1020F00081110CC08FEF809357020E94D40780910A
:102100007401811132C11092360237C10E94D40786
:1021100060905602772467FC7094F5E06F0E711C96
:10212000640C751CC301CCD2482F87FF04C04F77C5
:102130005524539401C0512C413030F0463008F4FE
:1021400060C2483009F45DC2712C80915502882329
:10215000A9F0552099F0E0919301E73024F087E051
:10216000809393010BC0EF5FE0939301FF27E7FD9E
:10217000F095E559FE4F809136028083109255020A
:1021800050E0FA013197E830F10508F090C0E65CC4
:10219000FF4F63C280916A0181111BC081E080936F
:1021A0006A0127EE271508F486C0E72DE695E69527
:1021B000E695F0E0E85CFD4F872D8770B80102C01E
:1021C000660F771F8A95E2F7CB019081892B808378
:1021D00072C010926A0177EE7715A0F0E72DE695B0
:1021E000E695E695F0E0E85CFD4F872D8770D80115
:1021F00002C0AA0FBB1F8A95E2F7CD01809590819E
:102200008923808382E00E940A0855C082E00E94F0
:102210000A08709236024FC082E00E940A0880913C
:10222000360287290EC082E00E940A0870948091CD
:102230003602872106C082E00E940A088091360299
:1022400087258093360237C081E00E940A0880917A
:10225000930187FD16C0E82FFF27E7FDF095E559AC
:10226000FE4F90819093360281500CC081E00E9415
:102270000A088091930187FD04C080916B018093CF
:1022800036028FEF8093930116C080917301811104
:1022900006C081E0809373017092B7020EC08091F6
:1022A000B70281110AC01092730182E001C081E07F
:1022B0000E940A0802C081E001C080E090913602CD
:1022C000909354025AC020915402232B209354021D
:1022D000322F32953F70322BE8E9F1E080E0DF01E8
:1022E00012979C91992309F440C0492F4695469531
:1022F000469550E09770DA01A85CBD4F6C9170E094
:10230000092E02C0759567950A94E2F760FF2FC009
:10231000DA01AA58BE4F4C9150E002C0559547953E
:102320009A95E2F740FD23C0DF0111979C91A081AF
:10233000BA2FB2236B2F70E0492F50E04095509593
:1023400046235723452B99F4492F42274A2359F016
:10235000B1110DC04A2F432351F0A92392959F70CC
:102360009A23941304C00E94F60780E006C08F5F92
:102370003596803209F0B3CFF8CF782C782AE1F186
:102380008091380283FF11C08091760183FD0DC0DA
:1023900080912603811105C00E940F090E941B092C
:1023A00004C0109226030E94C70180912603813049
:1023B00021F010F183508C30F8F43091B50220E018
:1023C000F60191916F01D7018D917D01981306C09F
:1023D0002F5F2A31A9F73093B5020EC0892B8927C8
:1023E000211101C0807F91E0930F882389F33FEF93
:1023F000380F8323392FF7CFE09126038E2F90E0FB
:10240000FC013297ED30F10508F067C0EE5BFF4F3D
:1024100024C180912B0380FF02C02D9A01C02D980A
:1024200080912B0381FF02C02E9A01C02E988091CB
:102430002B0382FF02C02C9A50C02C984EC00E94E1
:10244000DE0849E362E010C00E94DE0849E362E072
:1024500009C00E94DE0843E561E006C00E94DE0874
:1024600043E561E091E089270E94E5088823A9F10E
:1024700036C00E94DE08811105C02FC00E94DE0810
:1024800081112BC08091540282608093540225C038
:102490000E94DE08882331F081E017C00E94DE0828
:1024A0008823D1F31092750118C00E94DE0888239A
:1024B000C9F382E00AC00E94DE088111F3CFF9CF90
:1024C0000E94DE08882371F383E08093750105C0C4
:1024D0000E94DE088111E6CFF7CF772049F081E036
:1024E0008093030180930401809302018093010192
:1024F0008091910180FF07C09091530290FD03C02D
:102500001092750119C081FF06C09091530291FD90
:1025100002C081E00FC082FF06C09091530292FD7D
:1025200002C082E007C083FF07C08091530283FD91
:1025300003C083E0809375018091750190915202F0
:10254000977061F0ECE1F3E02191322F32953F700A
:10255000391302C0822F8F709E12F6CF90911B0309
:1025600089130E949D0880913403882321F0809173
:1025700034038530B9F58091B802882399F1E8E3F6
:10258000F2E020E041914423A1F080E090E050E0AF
:10259000BA01082E02C0759567950A94E2F760FFAC
:1025A00004C0322F380F343040F401968830910542
:1025B00079F7285F283E31F715C084E089BD86E0B1
:1025C00089BD09B400FEFDCF8091D8008F7D809336
:1025D000D8008091E00082608093E0008091E0006C
:1025E00081FDFCCF85E391E04AD885E291E047D8B0
:1025F00085E191E044D885E091E041D80E94CB0488
:10260000B4CCC301019649835BD0782E49819DCD1E
:102610000024552704C0080E591F880F991F0097E2
:1026200029F076956795B8F37105B9F7802D952F48
:102630000895AA1BBB1B51E107C0AA1FBB1FA61709
:10264000B70710F0A61BB70B881F991F5A95A9F75B
:1026500080959095BC01CD010895EE0FFF1F059068
:10266000F491E02D0994FB01DC0104C08D910190EF
:10267000801921F441505040C8F7881B990B0895E8
:10268000FB01DC0102C001900D9241505040D8F78F
:102690000895DC0101C06D9341505040E0F708956A
:1026A000DC01CB01FC01F999FECF06C0F2BDE1BD12
:1026B000F89A319600B40D9241505040B8F7089501
:1026C000F999FECF92BD81BDF89A992780B50895FA
:1026D000DC01A40FB51F4150504040F0CB01840FE6
:1026E000951F2E9105D041505040D8F70895262FC0
:1026F000F999FECF92BD81BDF89A019700B40216F8
:1027000039F01FBA20BD0FB6F894FA9AF99A0FBEA5
:062710000895F894FFCFCC
:10271600010101010103840800000100000300001B
:1027260000000000000282200000010000160000E8
:1027360000000000000183080000013503080000C6
:1027460000000000000081080000010000080000F1
:10275600000000000025206F6BF201D2016301F832
:1027660000290242025B0274025E00BA00160100F2
:00000001FF
